:020000040000FA
:100000008316FF23900005127B3081002730950076
:10001000831205120730990005080739820717284F
:100020003F2864288728A928CA28EA280C286400C1
:10003000851A1828851E1A281030A0000516000001
:1000400000000000000000000000000000000000B0
:100050000000000000000000000000000000051289
:100060000000000000000000000000000000000090
:100070000000000000000000A00B1E2817286400EC
:10008000851A4028851E42281130A0000516000060
:100090000000000000000000000000000000000060
:1000A0000000000000000000000005120000000039
:1000B0000000000000000000000000000000000040
:1000C0000000A00B46283F286400851A6528851E7D
:1000D00067281230A0000516000000000000000094
:1000E0000000000000000000000000000000000010
:1000F00000000512000000000000000000000000E9
:100100000000000000000000A00B6B2864286400C1
:10011000851A8828851E8A281230A000051600003E
:1001200000000000000000000000000000000000CF
:1001300000000000000000000512000000000000A8
:10014000000000000000000000000000A00B8E284E
:1001500087286400851AAA28851EAC281330A000C1
:100160000516000000000000000000000000000074
:100170000000000000000000000005120000000068
:100180000000000000000000000000000000A00BC4
:10019000B028A9286400851ACB28851ECD281430E4
:1001A000A000051600000000000000000000000094
:1001B0000000000000000000000000000512000028
:1001C0000000000000000000000000000000A00B84
:1001D000D128CA286400851AEB28851EED281C301A
:1001E000A000051600000000000000000000000054
:1001F00000000000051200000000000000000000E8
:06020000A00BF128EA2822
:02400E008C3FE5
:00000001FF
